:100000000C948A000C94A5000C94A5000C94A500F7
:100010000C94A5000C94A5000C94A5000C94A500CC
:100020000C94A5000C94A5000C94A5000C946107F9
:100030000C94A5000C9444020C94A5000C9473023B
:100040000C94A5000C94A5000C94A5000C94A5009C
:100050000C94A5001F1C1F1E1F1E1F1F1E1F1E1FEE
:100060002020202020202020202020202020202090
:10007000002043484F4F5345202F20454E544552B2
:1000800020002D2D2D2D2D2D2D2D2D2D2D2D2D2DDA
:100090002D2D0056657273696F6E202020312E3031
:1000A000320000454C4156523332202D20424153FC
:1000B000450000202020202020202020202020205B
:1000C00020200000000000000000000000000000F0
:1000D0000000005345542044415445202020202056
:1000E00020200000000000000000000000000000D0
:1000F0000000005345542054494D45202020202025
:1001000020200000000000000000000000000000AF
:100110000000000011241FBECFE5D8E0DEBFCDBF38
:1001200010E0A0E6B0E0E4ECFEE102C005900D9224
:10013000A43DB107D9F710E0A4EDB0E001C01D92D5
:10014000A03FB107E1F70C94050B0C9400000F934E
:100150001F93CF93DF938C01C0E0D0E0C817D9077D
:1001600038F48AE00E94BD002196C017D107C8F379
:10017000DF91CF911F910F91089520E02817A8F4E7
:1001800090E00000000000000000000000000000FF
:1001900000000000000000000000000000009F5F61
:1001A000943678F32F5F281758F3089590E0981746
:1001B00088F40000000000000000000000000000C3
:1001C00000000000000000000000000000009F5F31
:1001D000981778F30895BC01AC014F7050709C01E2
:1001E000207F3070F4E036952795FA95E1F7C90144
:1001F000E3E0880F991FEA95E1F7820F931F820FC2
:10020000931F480F591FCB0180709F70292F3327F0
:1002100084E690E0289FF001299FF00D389FF00DB3
:1002200011244E0F5F1F672F772762956F7088EE3E
:1002300093E0689F9001699F300D789F300D1124E5
:10024000420F531FCA0108950F931F938C012AE098
:1002500030E0B9010E94E20EFC01C801B9010E9420
:10026000E20E8B01CB01B9010E94E20E44E0880F3F
:10027000991F4A95E1F7E82BF92BC801B9010E94B3
:10028000E20E8B01CB01B9010E94E20E982F882764
:10029000E82BF92BC801B9010E94E20ECB01B9018C
:1002A0000E94E20E982F88279295907FE82BF92BD9
:1002B000CF011F910F910895FC01ED5AFF4F24913A
:1002C000029729F463707070672B09F42F5F822FF7
:1002D000992708951F93182FD998807F84608BBB2E
:1002E000D99A0000000000000000D99880E30E9425
:1002F000D6001295107F14601BBBD99A0000000035
:1003000000000000D99880E30E94D6001F91089554
:100310001F93182FD998807F8BBBD99A00000000BB
:1003200000000000D99880E30E94D6001295107F4B
:100330001BBBD99A0000000000000000D99880E3A0
:100340000E94D6001F910895CF93DF93EC0188811E
:10035000882341F02196882329F00E946A01888130
:100360008823C1F7DF91CF910895CF93DF93EC01FC
:10037000FC018491882349F02196882331F00E9462
:100380006A01FE0184918823B9F7DF91CF91089526
:1003900099278130910561F0823091051CF4892BF9
:1003A00071F00CC08230910529F0039729F006C046
:1003B000605C05C0605F03C0605B01C060E06068B6
:1003C000862F0E9488018DE20E94D600089581E068
:1003D0000E94880182E090E00E94A7000895CF93D8
:1003E000DF93DB98DA98D99882E390E00E94A70027
:1003F000C2E0D0E080E38BBBD99A0000000000008F
:100400000000D9988AE090E00E94A7002197D7FFCA
:10041000F1CF80E28BBBD99A000000000000000001
:10042000D9988AE090E00E94A70088E20E948801A3
:1004300085E090E00E94A7008EE00E94880182E0A3
:1004400090E00E94A70086E00E94880182E090E090
:100450000E94A700DA9ADF91CF910895CF93C82F19
:1004600082958F708A3010F4805D01C0895C0E9493
:100470006A018C2F8F708A3010F4805D01C0895C16
:100480000E946A01CF9108951F920F920FB60F92AA
:1004900011242F938F939F93EF93FF938CB18093AD
:1004A000D5008091E6008830A0F48091EB00209187
:1004B000E600820F912D911DFC012F5F2093E60035
:1004C000887F9370E81BF90BE652FF4F8091D500AF
:1004D0008083FF91EF919F918F912F910F900FBE8D
:1004E0000F901F9018951F920F920FB60F92112424
:1004F00053981092D9000F900FBE0F901F9018952F
:100500008091E6008823E1F357988091E6008150BE
:100510008093E6008091EB00E82FFF27E652FF4F23
:10052000E0818F5F8093EB008091EB00883010F0CA
:100530001092EB00579A8E2F99270895982F80914B
:10054000D9008130E1F3539A9CB981E08093D900BE
:1005500008951F93CF93DF93EC011991112359F064
:100560001A3019F48DE00E949E02812F0E949E0293
:1005700019911123A9F7DF91CF911F91089510923E
:10058000EB008091EB008093E6001092D90088ED9B
:100590008AB98FE589B986E880BD0895A89AA99A95
:1005A000A09AA19AA89AA99A08951F93CF93DF932E
:1005B000182FC7E0D0E086E00E94D600812F99274F
:1005C0000C2E02C0959587950A94E2F780FF02C031
:1005D000A99A01C0A99886E00E94D600A89A86E050
:1005E0000E94D60086E00E94D600A8982197D7FFE7
:1005F000E2CF86E00E94D600A99AA19886E00E94E8
:10060000D600A89A86E00E94D60086E00E94D60016
:1006100013B312700000A89886E00E94D600A19A39
:100620000000812F9927DF91CF911F910895EF92BC
:10063000FF920F931F93CF93DF93182F062FEA019A
:100640007901A99886E00E94D600A8981E7F812F84
:100650000E94D502882319F0A99800000AC0802FB3
:100660000E94D502882399F0A998000002C0A99899
:10067000000086E00E94D600A89A86E00E94D6007C
:10068000A99A86E00E94D6008EEF90E020C02197C4
:100690008FEFCF3FD80761F0F70181917F010E9472
:1006A000D502882321F72197FFEFCF3FDF07A1F77E
:1006B000A998000086E00E94D600A89A86E00E94D1
:1006C000D600A99A86E00E94D60080E090E0E6E09D
:1006D000CDB7DEB70C941D0FAF92BF92CF92DF92D1
:1006E000EF92FF921F93CF93DF93C82F162F7A01BB
:1006F000CC24DD245901A99886E00E94D600A89850
:100700008C2F8E7F0E94D502882319F0A9980000B3
:100710001DC0812F0E94D502882319F0A9980000DE
:1007200015C0A99A86E00E94D600A89A86E00E9489
:10073000D600A99886E00E94D600A898C1608C2FA8
:100740000E94D502882381F0A998000086E00E94CB
:10075000D600A89A86E00E94D600A99A86E00E9458
:10076000D6008EEF90E05CC0A99AA198CE14DF0469
:1007700008F047C010E0C7E0D0E086E00E94D60055
:10078000A89A86E00E94D60086E00E94D600110F4B
:1007900099991160A89886E00E94D6002197D7FF0A
:1007A000ECCFF50111935F010894C11CD11CA19AF3
:1007B0000000CE14DF0490F4A99886E00E94D600D1
:1007C000A89A86E00E94D60086E00E94D600A898EB
:1007D00086E00E94D600A19800000FC0A99A86E08A
:1007E0000E94D600A89A86E00E94D60086E00E9469
:1007F000D600A89886E00E94D600CE14DF0408F444
:10080000B9CFA998000086E00E94D600A89A86E099
:100810000E94D600A99A86E00E94D60080E090E06F
:10082000DF91CF911F91FF90EF90DF90CF90BF901D
:10083000AF900895A8E0B0E0E0E2F4E00C94020F7D
:100840008C01F62EFC01818192810E94EB009C01BB
:10085000AC0197FF02C04D5F5F4F4C7F241B350BEF
:100860002887F8018085898387818A8386818B83A5
:1008700085818C83822F992766E0880F991F6A955E
:10088000E1F72481282B2D838081992755E0880F5B
:10089000991F5A95E1F72381282B2E8384E88F83B3
:1008A00021E030E040E06F2DCE0107960E947F06E8
:1008B000482F8823D1F526E030E041E06F2DCE01AE
:1008C00001960E947F06482F882379F58F8321E0C7
:1008D00030E048E06F2DCE0107960E947F06482F3A
:1008E000882319F584E08F8321E030E06F2DCE015D
:1008F00007960E947F06482F8823B9F40F5F1F4F89
:1009000022E030E040E16F2DC8010E947F06482FB1
:10091000882359F421E030E042E16F2DCE010896A2
:100920000E947F06482F882319F0842F992702C040
:1009300080E090E0E5E028960C941E0FAF92BF9205
:10094000DF92EF92FF920F931F93CF93DF93CDB778
:10095000DEB728970FB6F894DEBF0FBECDBF7C017F
:10096000D62E21E030E040E0CE0107960E949F069F
:10097000882309F05AC08F8182FD03C08DEF90E07B
:1009800070C026E030E041E06D2DCE0101960E945E
:100990009F06882309F049C057010894A11CB11C87
:1009A00022E030E040E16D2DC5010E949F068823C2
:1009B000E1F521E030E042E16D2DCE0108960E9484
:1009C0009F06882391F59D819295969596959370B3
:1009D000092F11278885081B11090115110539F107
:1009E000988717FF02C00C5F1F4FF701818192812A
:1009F0000E94EB00080F191FC8010E942401F70193
:100A00008183928322E030E040E16D2DC5010E9498
:100A10007F06882351F421E030E042E16D2DCE01C4
:100A200008960E947F06882311F099271AC02E810C
:100A3000822F992775E0969587957A95E1F78770CB
:100A4000F70180832F7123838D818F7384838C8141
:100A500085838B8186838A8187838981808780E0F3
:100A600090E028960FB6F894DEBF0FBECDBFDF91A1
:100A7000CF911F910F91FF90EF90DF90BF90AF90BB
:100A80000895A7E0B0E0E7E4F5E00C94020F8C01D4
:100A9000F62E21E030E040E0CE0107960E949F064E
:100AA000482F8823B1F58F8182FD03C08DEF90E040
:100AB00035C04983F80187818A8386818B8385814C
:100AC0008C8384818D8383818E8326E030E049E0AE
:100AD0006F2DCE0101960E947F06482F8823C9F40E
:100AE00080EB8F8321E030E048E06F2DCE01079648
:100AF0000E947F06482F882361F484E08F8321E0E1
:100B000030E06F2DCE0107960E947F06482F882384
:100B100019F0842F992702C080E090E0E5E0279645
:100B20000C941E0FAF92BF92DF92EF92FF920F9341
:100B30001F93CF93DF93CDB7DEB729970FB6F89405
:100B4000DEBF0FBECDBF7C01D62E21E030E040E0FD
:100B5000CE0107960E949F06882311F0992779C03D
:100B60008F8182FD03C08DEF90E073C026E030E0FE
:100B700049E06D2DCE0101960E949F06882309F061
:100B800066C057010894A11CB11C22E030E040E18E
:100B90006D2DC5010E949F06882309F058C021E0F1
:100BA00030E042E16D2DCE0108960E949F06882319
:100BB00009F04DC021E030E045E06D2DCE010996F1
:100BC0000E949F06882309F042C0998592959695C8
:100BD00096959370092F11278885081B1109011517
:100BE000110529F1988717FF02C00C5F1F4FF7010D
:100BF000818192810E94EB00080F191FC8010E9499
:100C00002401F7018183928322E030E040E16D2DE1
:100C1000C5010E947F068823D1F421E030E042E143
:100C20006D2DCE0108960E947F06882381F4F7017E
:100C30001182128210828E818F7183838D818F73D6
:100C400084838C8185838B8186838A81878380E0FE
:100C500090E029960FB6F894DEBF0FBECDBFDF91AE
:100C6000CF911F910F91FF90EF90DF90BF90AF90C9
:100C70000895A1E0B0E0EFE3F6E00C94020F8C01E0
:100C8000F62E21E030E040E0CE01820F931F0E945B
:100C90009F06482F882351F58981282F332722FD6D
:100CA00003C08DEF90E027C021FD03C0F801408311
:100CB00020C081E0F8018083498321E030E048E0F2
:100CC0006F2DCE01820F931F0E947F06482F88232D
:100CD00069F484E0898321E030E06F2DCE01820F3A
:100CE000931F0E947F06482F882319F0842F99278D
:100CF00002C080E090E0E5E021960C941E0FCF92B8
:100D0000DF92EF92FF920F931F937C01C62ED42E99
:100D100089010E94CE029701A8016D2D8C2D0E94A1
:100D20001703882319F08EEF90E002C080E090E076
:100D30001F910F91FF90EF90DF90CF900895CF9289
:100D4000DF92EF92FF920F931F937C01C62ED42E59
:100D500089010E94CE029701A8016D2D8C2D0E9461
:100D60006C03882319F08FEF90E002C080E090E0E0
:100D70001F910F91FF90EF90DF90CF900895CF9249
:100D8000DF92EF92FF920F931F936C01062F142FA7
:100D900079010E94CE021C5E9601A701612F802F6F
:100DA0000E941703882319F08EEF90E002C080E0C4
:100DB00090E01F910F91FF90EF90DF90CF900895FA
:100DC000CF92DF92EF92FF920F931F936C01062F49
:100DD000142F79010E94CE021C5E9601A701612F9B
:100DE000802F0E946C03882319F08FEF90E002C0DF
:100DF00080E090E01F910F91FF90EF90DF90CF90F7
:100E0000089517B887EC86B9349BFECF84B195B1AD
:100E100023E0863B920788F523E08335920718F09C
:100E200087E390E0089522E08F3E920718F086E372
:100E300090E0089522E08B38920718F085E390E067
:100E4000089521E0853F920718F084E390E008952B
:100E500021E08F35920718F083E390E008958739F9
:100E6000910518F082E390E00895C39718F081E3AC
:100E700090E0089580E390E0089580E090E0089588
:100E8000CF930E940107C82F882381F08AE090E069
:100E90000E94A7000E9401078C1741F48AE090E0AD
:100EA0000E94A7000E9401078C1719F080E090E0D3
:100EB00006C00E9401078C17E1F38C2F9927CF9170
:100EC000089578941F920F920FB60F9211242F93CA
:100ED0003F938F939F938091D4008F5F8093D40032
:100EE0008091D400843208F48AC01092D40080919A
:100EF000E9009091EA0005969093EA008093E9005A
:100F00008091E9009091EA00885E93400CF477C0EC
:100F10001092EA001092E9008091EC009091ED00AF
:100F200001969093ED008093EC008091EC009091FD
:100F3000ED00CC970CF463C01092ED001092EC0021
:100F40008091E4009091E50001969093E5008093F4
:100F5000E4008091E4009091E500CC970CF44FC040
:100F60001092E5001092E4008091E7009091E80073
:100F700001969093E8008093E7008091E7009091BC
:100F8000E8004897E4F11092E8001092E7008091A1
:100F9000D6009091D70001969093D7008093D60009
:100FA0008091D800282F33278091D6009091D700C8
:100FB0002817390724F521E030E03093D70020933B
:100FC000D6008091E2009091E300820F931F9093EE
:100FD000E3008093E2008091E2009091E3000D979E
:100FE00074F03093E3002093E2008091EE00909142
:100FF000EF00820F931F9093EF008093EE009F917C
:101000008F913F912F910F900FBE0F901F901895C9
:10101000A9E0B0E0EEE0F8E00C94040F89B78E7F11
:1010200089BF8091D6009091D7000E9424018D83C2
:101030008091E2009091E3000E9424018C838091D2
:10104000EE009091EF000E9424018A839B8380919F
:10105000E7009091E8000E9424018E838091E400D3
:101060009091E5000E9424018F838091EC00909183
:10107000ED000E94240188878091E9009091EA00A8
:101080006AE070E00E94E20ECB010E942401898791
:1010900062EACE0101960E941A04182F60E0862FA2
:1010A0000E94C801112359F412BF82E083BF10933C
:1010B000D40089B7816089BF80E690E018C081E7DD
:1010C00090E00E94A40160E081E00E94C8011D3F01
:1010D00021F482E890E00E94A4011E3F21F483E9FC
:1010E00090E00E94A4011F3F21F484EA90E00E9456
:1010F000A40188EB9BE00E94A700E3E029960C94F2
:10110000200FA9E0B0E0E7E8F8E00C94040F89B7FD
:101110008E7F89BF62EACE0101960E949E04182F3D
:10112000882309F062C08D8199270E94EB0090937B
:10113000D7008093D6008C8199270E94EB00909372
:10114000E3008093E2008A819B810E94EB009093F0
:10115000EF008093EE008E8199270E94EB00909320
:10116000E8008093E7008F8199270E94EB0090931D
:10117000E5008093E400888599270E94EB00909316
:10118000ED008093EC00898599270E94EB009C017B
:10119000E3E0220F331FEA95E1F7280F391F280FEC
:1011A000391F3093EA002093E9008091E900909183
:1011B000EA00845E934024F01092EA001092E90065
:1011C0006091EE007091EF008091E2009091E30059
:1011D0000E945C018093D80012BF82E083BF10930D
:1011E000D40089B7816089BF22C060E0862F0E9449
:1011F000C80181E790E00E94A40160E081E00E94C4
:10120000C8011D3F21F482E890E00E94A4011E3F26
:1012100021F483E990E00E94A4011F3F21F484EAB5
:1012200090E00E94A40188EB9BE00E94A700E3E00D
:1012300029960C94200FDF92EF92FF920F931F9349
:10124000CF93F82E162FD42EE22E15C0612F8F2D9E
:101250000E94C801802F0E946A01612F8F2D0E9479
:10126000C801C73319F40E1508F40F5FC43319F41D
:10127000D01608F401500E944007C82F882331F38C
:10128000873321F3843311F3813319F480E090E044
:1012900002C0802F9927CF911F910F91FF90EF905F
:1012A000DF900895A2E1B0E0E8E5F9E00C94030FC7
:1012B0008091EE009091EF009F938F938091E200D8
:1012C0009091E3009F938F938091D6009091D700E7
:1012D0009F938F9385EB90E09F938F938E010F5F89
:1012E0001F4F1F930F930E94C10B60E082E00E948A
:1012F000C801C8010E94A4018091EC009091ED000A
:101300009F938F938091E4009091E5009F938F933A
:101310008091E7009091E8009F938F9384EC90E098
:101320009F938F931F930F930E94C10B60E083E004
:101330000E94C801C8010E94A4018DB79EB74496BF
:101340000FB6F8949EBF0FBE8DBFE4E062960C947A
:101350001F0FACE0B0E0EFEAF9E00C94FF0E0E9442
:10136000E7018091EE009091EF009F938F93809121
:10137000E2009091E3009F938F938091D60090912B
:10138000D7009F938F9385EB90E09F938F936E018F
:101390000894C11CD11CDF92CF920E94C10B60E067
:1013A00083E00E94C801C6010E94A40100E0102F42
:1013B000602F83E00E94C8018DB79EB70A960FB6D2
:1013C000F8949EBF0FBE8DBF4BC0013319F480E06F
:1013D00090E069C0063369F4112359F011501530BB
:1013E00009F414E0123009F411E0612F83E00E9447
:1013F000C801053369F4193058F41F5F123009F43D
:1014000013E0153009F416E0612F83E00E94C80153
:10141000073311F0043321F560E0862F0E94C801E4
:1014200081E790E00E94B5017601E10EF11CF70121
:10143000008129E340E3612F83E00E941B09882398
:1014400011F0F70180830E94E70160E083E00E94D1
:10145000C801C6010E94A401612F83E00E94C80157
:101460000E944007082F803309F0AFCF1B821E82F5
:101470001B86CE0101960E948C0B9093D70080931F
:10148000D600CE0104960E948C0B9093E3008093CB
:10149000E200CE0107960E948C0B9093EF008093A0
:1014A000EE0081E090E0E8E02C960C941B0FACE09D
:1014B000B0E0EDE5FAE00C94FF0E0E94E7018091A8
:1014C000EC009091ED009F938F938091E4009091B8
:1014D000E5009F938F938091E7009091E8009F93A0
:1014E0008F9384EC90E09F938F936E010894C11CBE
:1014F000D11CDF92CF920E94C10B60E083E00E947A
:10150000C801C6010E94A40100E0102F602F83E0F3
:101510000E94C8018DB79EB70A960FB6F8949EBF79
:101520000FBE8DBF4BC0013319F480E090E069C05D
:10153000063369F4112359F01150153009F414E001
:10154000123009F411E0612F83E00E94C8010533D5
:1015500069F4173058F41F5F123009F413E01530A6
:1015600009F416E0612F83E00E94C801073311F0EF
:10157000043321F560E0862F0E94C80181E790E0E6
:101580000E94B5017601E10EF11CF701008129E30B
:1015900040E3612F83E00E941B09882311F0F701CB
:1015A00080830E94E70160E083E00E94C801C601D9
:1015B0000E94A401612F83E00E94C8010E9440079D
:1015C000082F803309F0AFCF1B821E821986CE010F
:1015D00001960E948C0B9093E8008093E700CE0167
:1015E00004960E948C0B9093E5008093E400CE015A
:1015F00007960E948C0B9093ED008093EC0081E0A5
:1016000090E0E8E02C960C941B0FCFE5D8E0DEBF0D
:10161000CDBF8EEF8ABB1BBA83E085BB84BB82E063
:1016200081BB0E94EF010E94E70183EA90E00E94E3
:10163000B50160E081E00E94C80183E990E00E946A
:10164000B5010E9481087894E090EC00F090ED00E4
:10165000C0E0D0E00E944007182F882309F44DC055
:1016600060E081E00E94C80182E890E00E94B5013C
:101670001233A1F42196C330D10514F0C0E0D0E0BC
:1016800060E0862F0E94C801CE01A5E0880F991F57
:10169000AA95E1F78D549F4F0E94B501103369F56B
:1016A0000E94E701C130D10539F0C230D105CCF03C
:1016B000C230D10539F015C089B78E7F89BF0E942D
:1016C000A90905C089B78E7F89BF0E94570A892B57
:1016D00019F00E94080803C089B7816089BFC0E083
:1016E000D0E00E94E701CE01F5E0880F991FFA953E
:1016F000E1F78D549F4F0E94B5018091EC009091CD
:10170000ED00E816F90609F4A5CFE090EC00F090A2
:10171000ED000E9452099ECFFC0188279927E8948A
:1017200021912223F1F02032D9F32930C9F32A3054
:10173000B9F32C30A9F32D3099F3263789F32B32E6
:1017400019F02D3221F468942191222351F0203395
:1017500044F02A3334F420530E94B90B820F911DB8
:10176000F3CF8115910521F01EF480959095019697
:1017700008957AE0979F902D879F802D910D1124D9
:1017800008950F931F93CF93DF93CDB7DEB72C97B8
:101790000FB6F894DEBF0FBECDBF0B891C89ED8953
:1017A000FE8936E03C8309831A834FEF5FE74D8360
:1017B0005E83AE01495E5F4FBF01CE0101960E947C
:1017C000F20B2F813885020F131FD8011C922C9623
:1017D0000FB6F894DEBF0FBECDBFDF91CF911F9142
:1017E0000F9108952F923F924F925F926F927F9246
:1017F0008F929F92AF92BF92CF92DF92EF92FF9221
:101800000F931F93CF93DF93CDB7DEB762970FB6D9
:10181000F894DEBF0FBECDBFAA24BB2465014C01E6
:101820006D877E874F87588B44245524FC01468260
:101830005782838181FD63C28FEF9FEF77C240FEA5
:101840004CC2862D80538A30E0F4F0E36F1641F4E9
:101850002A89222329F4772019F480E091E08BC0B3
:101860008AE09A89989F902D1124892F860D8053A4
:101870008A8B882314F4EFE7EA8B43FC40C27A8812
:101880003EC243FE05C0FA89FF2311F421E02A8BF2
:10189000862D992787FD90958836910554F58536D4
:1018A00091050CF06BC08835910509F4DBC08935D2
:1018B0009105B4F48B32910509F442C08C32910544
:1018C00044F48032910509F43FC0839709F442C083
:1018D000FAC18D329105D9F18E9709F440C0F3C158
:1018E0008336910509F454C08436910509F480C00B
:1018F000EAC18037910509F4ADC08137910584F4C0
:101900008C369105B1F18D3691052CF4893691050F
:1019100009F46EC0D8C18F36910509F498C0D3C1BF
:101920008537910509F4A0C08637910524F48337E3
:101930009105B9F1C8C18837910509F493C0C3C1B5
:1019400080E190E0482A592AE0E2F0E005C080E812
:1019500090E011C0E0E4F0E04E2A5F2AD0C188E0B8
:1019600090E0482A592AEFEFFEEF4E225F221A8AB2
:10197000C6C184E090E0482A592AC1C10F2EFFE376
:10198000AF2EF02D7A940F2EF3E66F2EF02D42C17C
:10199000EF85F889CF0102968F87988BA0807A9483
:1019A00039C1EF85F889CF0102968F87988BA08087
:1019B000B180198AF5018081882349F099899F5F58
:1019C000998BF501E90FF11D80818823B9F743FE5A
:1019D0000CC04A89242F332727FD3095E9898E2FA3
:1019E0009927281739070CF4498BF9897F1A12C1F6
:1019F00042FE0BC0EF85F889CF0104968F87988B44
:101A000020813181428153810DC0EF85F889CF015A
:101A100002968F87988B808191819C01442737FDA6
:101A20004095542F59016A01552364F4E2E0F0E037
:101A30004E2A5F2AD094C094B094A094A11CB11CEB
:101A4000C11CD11C8FEB9FEF482259222BC098E07C
:101A5000998B0AC0E0E4F0E04E2A5F2A0F2EF8E7E7
:101A60006F2EF02DF0E1F98B42FE0BC0EF85F88967
:101A7000CF0104968F87988B2081318142815381D9
:101A80000BC0EF85F889CF0102968F87988B8081F4
:101A900091819C014427552759016A01EFECFFEF22
:101AA0004E225F221E010894211C311CF989EF2E61
:101AB000FF2400271127C601B501A80197010E9444
:101AC000400FDC01CB01F10180838A301CF0860DD0
:101AD000815203C0F1018081805DF10181931F017A
:101AE000C601B501A80197010E94400F59016A0182
:101AF0002115310541055105F1F6CE010196A22CC3
:101B0000A81AC20182739070892B09F07A9446FE5C
:101B10000FC0872D992787FD9095F989F03131F411
:101B20000F2EFEEF7F2EF02D780E02C0782E7A94C5
:101B300043FE12C04A89242F332727FD30958A2D72
:101B40009927821793072CF087EF9FEF482259229D
:101B500003C09A899A199A8B43FE03C0EA897E1AB8
:101B600001C07A18C20180789170892B69F4872DA1
:101B70007A9418164CF4B40180E290E00E94AF0E03
:101B8000872D7A941816BCF341FE04C0B4018DE28F
:101B900090E00BC044FE04C0B4018BE290E005C0AD
:101BA00045FE05C0B40180E290E00E94AF0E46FE03
:101BB0000FC0B40180E390E00E94AF0EF989F031CC
:101BC00039F4862D992787FD9095B4010E94AF0EB8
:101BD00050FE0DC0872D7A9418164CF4B40180E3A2
:101BE00090E00E94AF0E872D7A941816BCF343FE46
:101BF00011C08A89282F21502A8B18165CF4B40151
:101C000080E390E00E94AF0E8A89482F41504A8BB2
:101C10001816ACF3842D807869F4872D7A94181601
:101C20004CF4B40180E290E00E94AF0E872D7A94CC
:101C30001816BCF383E6681641F48A2D992787FDB0
:101C40009095B4010E94AF0E2DC093E76916B1F4D0
:101C5000E989E150E98BEF3F29F1F501808199276E
:101C600087FD90950894A11CB11CB4010E94AF0E91
:101C7000F989F150F98BFF3F81F714C0CE0101962D
:101C80002816390679F08E010F5F1F4FF1018291FE
:101C90001F01992787FD9095B4010E94AF0E201671
:101CA0003106A1F7842D8078A9F0872D7A94181633
:101CB0008CF4B40180E290E00E94AF0E872D7A94FC
:101CC0001816BCF307C0862D992787FD9095B4019F
:101CD0000E94AF0E4424552412C0F5E26F1641F461
:101CE0004424552443941A8A7A882AE0298B07C011
:101CF000862D992787FD9095B4010E94AF0EF401BF
:101D0000838183FF08C0ED85FE85CF0101968D8715
:101D10009E87649005C0ED85FE856190ED87FE8706
:101D2000662009F08CCDF4018681978162960FB60A
:101D3000F894DEBF0FBECDBFDF91CF911F910F9101
:101D4000FF90EF90DF90CF90BF90AF909F908F90DB
:101D50007F906F905F904F903F902F9008950F93DA
:101D60001F93CF93DF938C01EB018B81992781FF28
:101D700022C082FF14C02E813F814C815D812417D7
:101D800035073CF4A881B9810D93A883B9832E81CE
:101D90003F812F5F3F4F2E833F83C8010EC0E885F0
:101DA000F985802F0995892B31F4EE81FF813196D9
:101DB000EE83FF83F2CF8FEF9FEFDF91CF911F91E3
:101DC0000F91089597FB092E07260AD077FD04D0BE
:101DD00043D006D000201AF4709561957F4F089586
:101DE000F6F7909581959F4F08952F923F924F92CD
:101DF0005F926F927F928F929F92AF92BF92CF929B
:101E0000DF92EF92FF920F931F93CF93DF93CDB7A3
:101E1000DEB7CA1BDB0B0FB6F894DEBF0FBECDBF1B
:101E200009942A88398848885F846E847D848C84EC
:101E30009B84AA84B984C884DF80EE80FD800C81F5
:101E40001B81AA81B981CE0FD11D0FB6F894DEBFD8
:101E50000FBECDBFED010895AA1BBB1B51E107C00A
:101E6000AA1FBB1FA617B70710F0A61BB70B881F2A
:101E7000991F5A95A9F780959095BC01CD010895B9
:101E8000A1E21A2EAA1BBB1BFD010DC0AA1FBB1F7E
:101E9000EE1FFF1FA217B307E407F50720F0A21BF0
:101EA000B30BE40BF50B661F771F881F991F1A945D
:101EB00069F760957095809590959B01AC01BD0187
:041EC000CF010895B1
:101EC40053455420525443204F4B2020202020209F
:101ED40000525443202D204552524F52202020209E
:101EE40020004E4F5420494E495449414C495A45CB
:101EF40044200057524954454552524F5220202005
:101F040020202000524541444552524F5220202067
:101F14002020202000253032642E253032642E25E6
:101F240030346400253032643A253032643A253046
:041F34003264000013
:00000001FF
